:1000000033C000004CC000004AC0000048C00000DF
:1000100046C0000044C0000042C0000040C00000D4
:100020003EC000003CC000003AC0000038C00000E4
:1000300036C0000034C0000032C0000030C00000F4
:100040002EC000002CC00000AFC0000028C000007F
:1000500026C0000024C0000022C0000020C0000014
:100060001EC000001CC0000011241FBECFEFD4E052
:10007000DEBFCDBF11E0A0E0B1E0E2E0F4E002C0FD
:1000800005900D92AC37B107D9F711E0ACE7B1E0BC
:1000900001C01D92A139B107E1F723D1B0C1B0CFA2
:1000A0008EBD0DB407FEFDCF0895CF93C82F982FB6
:1000B00092959F709A3010F480E301C087E3890F16
:1000C000EFDF8C2F8F708A3010F4805D01C0895C67
:1000D000CF91E6CFE5DF80E090E00895FC0121912B
:1000E000CF01222369F03091C00035FFFCCFE7EB50
:1000F000FBE03197F1F700C000002093C600EECF7F
:10010000089598E028E02A95F1F787FF02C05798F4
:1001100001C0579A880F28E02A95F1F7569820E1F8
:100120002A95F1F7569A915069F7579880E18A9588
:10013000F1F7569890E19A95F1F789B1569A28E02F
:100140002A95F1F7881F8827881F0895579A569A8D
:1001500088E08A95F1F7569888E08A95F1F75798E4
:100160000895CF93DF93D82FC62F9BB19F739BB970
:100170009AB19F739AB9579A88E08A95F1F7569A7F
:1001800080E4BFDF81110BC08D2FBBDF811107C061
:100190008C2FB7DF811103C0D9DF80E002C0D6DF2A
:1001A00081E0DF91CF9108951F920F920FB60F92C9
:1001B00011242F933F934F935F936F937F938F936C
:1001C0009F93AF93BF93EF93FF93CF93DF93CDB7FD
:1001D000DEB72897DEBFCDBF8091C600888780E05C
:1001E0005FDF88855DDF80918A01882309F460C024
:1001F00080918701909188018A30910560F49C017B
:100200002F5F3F4F30938801209387012885FC01A1
:10021000E358FE4F208388858A3021F088858E320E
:1002200009F046C08091870190918801029721F0E2
:1002300082E591E053DF38C080917D0197E0EEE0E8
:10024000F1E0DE01119601900D929A95E1F790EDA3
:10025000980F983070F4292F81E090E0022E01C0B1
:10026000880F0A94EAF790917C01982B90937C0177
:1002700005C08F7D8F3411F410927C0180917C0138
:10028000982F92959F709F599B838F708F598C8365
:10029000CE01019623DF60917C0170E089E090E05F
:1002A00060DF03DF8AE0FCDE109288011092870194
:1002B00028960FB6F894DEBF0FBECDBFDF91CF9169
:1002C000FF91EF91BF91AF919F918F917F916F912E
:1002D0005F914F913F912F910F900FBE0F901F9004
:1002E00018955D98559AF89484B1837D84B9249AC1
:1002F00080E48CBD80E091E090938E0180938D012D
:1003000078945D9A87EB9BE00197F1F700C00000BD
:1003100080E0C6DE60E070E080E090E022DFC5DED5
:100320008AE0BEDE6AEA70E089E090E01ADFBDDEB6
:100330008AE0B6DE8BE990E09093C5008093C4001C
:1003400082E08093C00088E98093C10086E08093BA
:10035000C200519A3D9A45988FE295E70197F1F7CF
:1003600000C00000459A9FEF22E587E091502040B1
:100370008040E1F700C0000085E191E0AFDE9FEF33
:1003800022E587E0915020408040E1F700C0000066
:1003900080E291E0A3DE9FEF22E587E091502040CC
:1003A0008040E1F700C0000085E291E097DE9FEF1A
:1003B00022E587E0915020408040E1F700C0000036
:1003C0008AE391E08BDE9FEF22E587E091502040A9
:1003D0008040E1F700C0000085E491E07FDE789482
:1003E0009FEF22E587E0915020408040E1F700C078
:1003F000000081E080938A0180918901FDCFF8940B
:02040000FFCF2C
:1004020000000002000000006A00000000003A3A0A
:10041200003A3A0A0041542B52657365740D0A0082
:1004220041540D0A0041542B4E414D4546616972BB
:100432006C616E653530300D0A0041542B524F4CC1
:1004420045300D0A0041542B50494E353536350D95
:100452000A0042616420666F726D61742E204E65DF
:100462006564204E756D626572206F7220274F277A
:0C04720020666F72206F66662E0A000084
:00000001FF
